:020000040000FA
:020000002428B2
:08000800F0000308F10083126F
:100010000B190D280B1816281F280B11C014C10B23
:100020001F2840150A30C100C20A1F280B10851D69
:100030001F28C4191F2843148316960183127108C0
:100040008300F00E700E090083018B0185010730DB
:10005000990083162830850040308F0008309600C4
:100060000830810083128101A8308B00C401C301D4
:10007000C5010A30C100401940204318B3203B2875
:100080004011C418482844194A28C4194C284D283E
:100090004E204D2860204D28A02008000930420243
:1000A000031D5B2805125C200430C400050883167C
:1000B0000830960083120800C2010A30C10008000F
:1000C0003C304202031C9F288316960183120530A0
:1000D00045020130031991280B3045020230031903
:1000E0009128173045020430031991280430450245
:1000F0000730031991280D30450201300319952866
:100100001B30450202300319952837304502043070
:10011000031995280C3045020730031995285C20F7
:100120009C2805040739C600982805050506C60061
:100130003830050546048500C5010830C4000800B4
:1001400005304202031CB228051205088316083048
:100150009600831263000230C40083169601831256
:10016000C501B3200800431005164419BD205C20CA
:10017000C419BC280230C400080003304202031C2A
:10018000D428333042020318D42815304202031C0D
:10019000CE281E3042020318D128D4280314C50DDE
:1001A000D7280310C50DD7285C200830C4000800EC
:02400E00C43CB0
:00000001FF
